:020000040800F2
:10000000600600206D010008470300081503000882
:100010004503000827020008A504000800000000AE
:10002000000000000000000000000000990300082C
:1000300029020008000000004903000851040008DC
:100040008701000887010008870100088701000870
:100050008701000887010008870100088701000860
:100060008701000887010008870100088701000850
:100070008701000887010008870100088701000840
:100080008701000887010008870100088701000830
:100090008701000887010008870100088701000820
:1000A0008701000887010008870100088701000810
:1000B0008701000887010008870100088701000800
:1000C00087010008870100088701000887010008F0
:1000D00087010008870100088701000887010008E0
:1000E00087010008870100088701000800F002F876
:1000F00000F02CF80AA090E8000C82448344AAF196
:100100000107DA4501D100F021F8AFF2090EBAE893
:100110000F0013F0010F18BFFB1A43F0010318473B
:100120008C0300009C03000000230024002500260F
:10013000103A28BF78C1FBD8520728BF30C148BF4A
:100140000B6070471FB51FBD10B510BD00F031F832
:100150001146FFF7F7FF00F0A6F900F04FF803B4DF
:10016000FFF7F2FF03BC00F057F800000948804792
:1001700009480047FEE7FEE7FEE7FEE7FEE7FEE789
:10018000FEE7FEE7FEE7FEE704480549054A064BA1
:100190007047000055040008ED00000860000020D2
:1001A0006006002060020020600200207047704757
:1001B0007047754600F02CF8AE4605006946534678
:1001C00020F00700854618B020B5FFF7DDFFBDE839
:1001D00020404FF000064FF000074FF000084FF0AE
:1001E000000B21F00701AC46ACE8C009ACE8C0093F
:1001F000ACE8C009ACE8C0098D46704710B50446AC
:10020000AFF300802046BDE81040FFF7A8BF000014
:10021000004870470000002001491820ABBEFEE7EF
:10022000260002007047FEE7704700B502464FF413
:100230007A7302E0184600F004F8521E501CF9D1FF
:1002400000BD00EBC000C1004FF0E0204161002183
:100250008161052101610169C903FCD504210161A6
:1002600070472DE9F0410022CC7804F00F03E4063A
:1002700001D58C7823430C784FF00F0714F0FF0F53
:100280004FF0010C1CD005680CFA02F40E882640D1
:10029000A64211D1960007FA06F825EA080503FAE6
:1002A00006F848EA0505CE78282E02D0482E02D05E
:1002B00002E0446100E00461521C082AE4D30560B6
:1002C0000A88FF2A1ED94568002202F108060CFAA6
:1002D00006F40E882640A64210D1960007FA06F8CA
:1002E00025EA080503FA06F848EA0505CE78282E1F
:1002F00000D14461CE78482E00D10461521C082AF6
:10030000E3D34560BDE8F081002A01D00161704768
:1003100041617047FEE7000008B50121042000F0AC
:1003200015F810208DF803004020ADF800000320E0
:100330008DF8020069460248FFF793FF08BD0000F0
:1003400000080140FEE7704770470000054A002999
:1003500003D0916901439161704791698143916133
:100360007047000000100240FFF7D6FF094D4FF420
:10037000FA74012240212846FFF7C6FF2046FFF706
:1003800054FF002240212846FFF7BEFF2046FFF71A
:100390004CFFEEE700080140704700F001B8000094
:1003A0000CB50022019200922748016841F4803187
:1003B00001604FF4A063016801F4003100910199DC
:1003C000491C0191009911B901999942F3D1016831
:1003D000890302D50121009100E0009200990129D2
:1003E00030D11A490A6842F010020A600A6822F005
:1003F00003020A600A6842F002020A604168416032
:1004000041684160416841F480614160416821F484
:100410007C114160416841F4E8114160016841F09C
:100420008071016001688901FCD5416821F00301F8
:100430004160416841F0020141604168C1F38101BE
:100440000229FAD10CBD0000001002400020024039
:100450007047000010B50F48016841F001010160CC
:1004600041680D4A1140416001680C4A1140016029
:10047000016821F480210160416821F4FE0141609E
:100480004FF41F018160FFF788FF05494FF00060BE
:10049000086010BD001002400000FFF8FFFFF6FEEC
:1004A00008ED00E0FEE7FFF75FFFFCE7BC04000893
:0C04B00000000020600600002801000889
:04000005080000ED02
:00000001FF
